 allthr01

 Timestamp is 65b7cf49 (reproducible build file hash)

 Preferred load address is 0000000180000000

 Start         Length     Name                   Class
 0001:00000000 00001cc0H .text$mn                CODE
 0001:00001cc0 00000036H .text$mn$00             CODE
 0001:00001cf6 00000092H .text$x                 CODE
 0002:00000000 00000198H .idata$5                DATA
 0002:00000198 00000038H .00cfg                  DATA
 0002:000001d0 00000008H .CRT$XCA                DATA
 0002:000001d8 00000008H .CRT$XCZ                DATA
 0002:000001e0 00000008H .CRT$XIA                DATA
 0002:000001e8 00000008H .CRT$XIC                DATA
 0002:000001f0 00000008H .CRT$XIZ                DATA
 0002:000001f8 00000008H .CRT$XLA                DATA
 0002:00000200 00000008H .CRT$XLZ                DATA
 0002:00000208 00000008H .CRT$XPA                DATA
 0002:00000210 00000008H .CRT$XPZ                DATA
 0002:00000218 00000008H .CRT$XTA                DATA
 0002:00000220 00000010H .CRT$XTZ                DATA
 0002:00000228 00000000H .gehcont$y              DATA
 0002:00000228 00000000H .gfids$y                DATA
 0002:00000230 00000cd0H .rdata                  DATA
 0002:00000f00 00000000H .rdata$CastGuardVftablesA DATA
 0002:00000f00 00000000H .rdata$CastGuardVftablesC DATA
 0002:00000f00 00000028H .rdata$T                DATA
 0002:00000f28 00000064H .rdata$voltmd           DATA
 0002:00000f8c 0000031cH .rdata$zzzdbg           DATA
 0002:000012a8 00000008H .rtc$IAA                DATA
 0002:000012b0 00000008H .rtc$IZZ                DATA
 0002:000012b8 00000008H .rtc$TAA                DATA
 0002:000012c0 00000008H .rtc$TZZ                DATA
 0002:000012c8 00000004H .tls                    DATA
 0002:000012cc 00000004H .tls$                   DATA
 0002:000012d0 00000008H .tls$ZZZ                DATA
 0002:000012d8 00000218H .xdata                  DATA
 0002:000014f0 000000d8H .edata                  DATA
 0002:000015c8 00000064H .idata$2                DATA
 0002:0000162c 00000014H .idata$3                DATA
 0002:00001640 00000198H .idata$4                DATA
 0002:000017d8 00000440H .idata$6                DATA
 0003:00000000 00000170H .data                   DATA
 0003:00000170 00000668H .bss                    DATA
 0004:00000000 000002acH .pdata                  DATA

  Address         Publics by Value              Rva+Base               Lib:Object

 0000:00000000       __AbsoluteZero             0000000000000000     <absolute>
 0000:00000000       ___safe_se_handler_count   0000000000000000     <absolute>
 0000:00000000       ___safe_se_handler_table   0000000000000000     <absolute>
 0000:00000000       __arm64x_extra_rfe_table   0000000000000000     <absolute>
 0000:00000000       __arm64x_extra_rfe_table_size 0000000000000000     <absolute>
 0000:00000000       __arm64x_native_entrypoint 0000000000000000     <absolute>
 0000:00000000       __arm64x_redirection_metadata 0000000000000000     <absolute>
 0000:00000000       __arm64x_redirection_metadata_count 0000000000000000     <absolute>
 0000:00000000       __dynamic_value_reloc_table 0000000000000000     <absolute>
 0000:00000000       __enclave_config           0000000000000000     <absolute>
 0000:00000000       __guard_check_icall_a64n_fptr 0000000000000000     <absolute>
 0000:00000000       __guard_eh_cont_count      0000000000000000     <absolute>
 0000:00000000       __guard_eh_cont_table      0000000000000000     <absolute>
 0000:00000000       __guard_fids_count         0000000000000000     <absolute>
 0000:00000000       __guard_fids_table         0000000000000000     <absolute>
 0000:00000000       __guard_iat_count          0000000000000000     <absolute>
 0000:00000000       __guard_iat_table          0000000000000000     <absolute>
 0000:00000000       __guard_longjmp_count      0000000000000000     <absolute>
 0000:00000000       __guard_longjmp_table      0000000000000000     <absolute>
 0000:00000000       __hybrid_auxiliary_iat     0000000000000000     <absolute>
 0000:00000000       __hybrid_auxiliary_iat_copy 0000000000000000     <absolute>
 0000:00000000       __hybrid_code_map          0000000000000000     <absolute>
 0000:00000000       __hybrid_code_map_count    0000000000000000     <absolute>
 0000:00000000       __x64_code_ranges_to_entry_points 0000000000000000     <absolute>
 0000:00000000       __x64_code_ranges_to_entry_points_count 0000000000000000     <absolute>
 0000:00000100       __guard_flags              0000000000000100     <absolute>
 0000:00000000       __ImageBase                0000000180000000     <linker-defined>
 0001:00000000       ?NewObject@JNIEnv_@@QEAAPEAV_jobject@@PEAV_jclass@@PEAU_jmethodID@@ZZ 0000000180001000 f i liballthr01.obj
 0001:00000028       ?TranslateError@@YAPEBDW4jvmtiError@@@Z 0000000180001028 f   liballthr01.obj
 0001:00000348       ?create_raw_monitor@@YAPEAU_jrawMonitorID@@PEAU_jvmtiEnv@@PEBD@Z 0000000180001348 f   liballthr01.obj
 0001:000004bc       Agent_OnLoad               00000001800014bc f   liballthr01.obj
 0001:000005bc       Java_allthr01_checkInfo0   00000001800015bc f   liballthr01.obj
 0001:000005c4       Java_allthr01_startAgentThread 00000001800015c4 f   liballthr01.obj
 0001:000006c4       Java_allthr01_stopAgentThread 00000001800016c4 f   liballthr01.obj
 0001:00000780       __local_stdio_printf_options 0000000180001780 f i liballthr01.obj
 0001:00000788       check_info                 0000000180001788 f   liballthr01.obj
 0001:00000a18       create_jthread             0000000180001a18 f   liballthr01.obj
 0001:00000ac0       printf                     0000000180001ac0 f i liballthr01.obj
 0001:00000d1c       _Init_thread_footer        0000000180001d1c f   MSVCRT:thread_safe_statics.obj
 0001:00000d7c       _Init_thread_header        0000000180001d7c f   MSVCRT:thread_safe_statics.obj
 0001:00000de4       _Init_thread_notify        0000000180001de4 f   MSVCRT:thread_safe_statics.obj
 0001:00000e28       _Init_thread_wait          0000000180001e28 f   MSVCRT:thread_safe_statics.obj
 0001:00000e8c       __GSHandlerCheck           0000000180001e8c f   MSVCRT:gshandler.obj
 0001:00000eac       __GSHandlerCheckCommon     0000000180001eac f   MSVCRT:gshandler.obj
 0001:00000f20       __security_check_cookie    0000000180001f20 f   MSVCRT:amdsecgs.obj
 0001:00001260       _DllMainCRTStartup         0000000180002260 f   MSVCRT:dll_dllmain.obj
 0001:000012a0       __scrt_acquire_startup_lock 00000001800022a0 f   MSVCRT:utility.obj
 0001:000012dc       __scrt_dllmain_after_initialize_c 00000001800022dc f   MSVCRT:utility.obj
 0001:00001310       __scrt_dllmain_before_initialize_c 0000000180002310 f   MSVCRT:utility.obj
 0001:00001328       __scrt_dllmain_crt_thread_attach 0000000180002328 f   MSVCRT:utility.obj
 0001:00001350       __scrt_dllmain_crt_thread_detach 0000000180002350 f   MSVCRT:utility.obj
 0001:00001368       __scrt_dllmain_exception_filter 0000000180002368 f   MSVCRT:utility.obj
 0001:000013c8       __scrt_dllmain_uninitialize_c 00000001800023c8 f   MSVCRT:utility.obj
 0001:000013f8       __scrt_dllmain_uninitialize_critical 00000001800023f8 f   MSVCRT:utility.obj
 0001:0000140c       __scrt_initialize_crt      000000018000240c f   MSVCRT:utility.obj
 0001:00001458       __scrt_initialize_onexit_tables 0000000180002458 f   MSVCRT:utility.obj
 0001:000014e4       __scrt_is_nonwritable_in_current_image 00000001800024e4 f   MSVCRT:utility.obj
 0001:0000157c       __scrt_release_startup_lock 000000018000257c f   MSVCRT:utility.obj
 0001:000015a0       __scrt_uninitialize_crt    00000001800025a0 f   MSVCRT:utility.obj
 0001:000015cc       _onexit                    00000001800025cc f   MSVCRT:utility.obj
 0001:00001608       atexit                     0000000180002608 f   MSVCRT:utility.obj
 0001:00001620       __crt_debugger_hook        0000000180002620 f   MSVCRT:utility_desktop.obj
 0001:00001628       __scrt_fastfail            0000000180002628 f   MSVCRT:utility_desktop.obj
 0001:00001774       _guard_check_icall_nop     0000000180002774 f i MSVCRT:guard_support.obj
 0001:00001778       __raise_securityfailure    0000000180002778 f   MSVCRT:gs_report.obj
 0001:000017ac       __report_gsfailure         00000001800027ac f   MSVCRT:gs_report.obj
 0001:000018f4       __security_init_cookie     00000001800028f4 f   MSVCRT:gs_support.obj
 0001:000019a0       DllMain                    00000001800029a0 f   MSVCRT:dll_dllmain_stub.obj
 0001:000019c4       ?__scrt_initialize_type_info@@YAXXZ 00000001800029c4 f   MSVCRT:tncleanup.obj
 0001:000019d4       ?__scrt_uninitialize_type_info@@YAXXZ 00000001800029d4 f   MSVCRT:tncleanup.obj
 0001:000019e0       __local_stdio_scanf_options 00000001800029e0 f i MSVCRT:default_local_stdio_options.obj
 0001:000019e8       __scrt_initialize_default_local_stdio_options 00000001800029e8 f   MSVCRT:default_local_stdio_options.obj
 0001:00001a04       __scrt_get_dyn_tls_init_callback 0000000180002a04 f   MSVCRT:dyn_tls_init.obj
 0001:00001a0c       _RTC_Initialize            0000000180002a0c f   MSVCRT:initsect.obj
 0001:00001a48       _RTC_Terminate             0000000180002a48 f   MSVCRT:initsect.obj
 0001:00001a84       __isa_available_init       0000000180002a84 f   MSVCRT:cpu_disp.obj
 0001:00001c30       _get_startup_argv_mode     0000000180002c30 f   MSVCRT:argv_mode.obj
 0001:00001c38       __scrt_is_ucrt_dll_in_use  0000000180002c38 f   MSVCRT:ucrt_detection.obj
 0001:00001c50       memset                     0000000180002c50 f   vcruntime:VCRUNTIME140.dll
 0001:00001c56       __C_specific_handler       0000000180002c56 f   vcruntime:VCRUNTIME140.dll
 0001:00001c5c       __std_type_info_destroy_list 0000000180002c5c f   vcruntime:VCRUNTIME140.dll
 0001:00001c62       strcmp                     0000000180002c62 f   ucrt:api-ms-win-crt-string-l1-1-0.dll
 0001:00001c68       strlen                     0000000180002c68 f   ucrt:api-ms-win-crt-string-l1-1-0.dll
 0001:00001c6e       _initterm                  0000000180002c6e f   ucrt:api-ms-win-crt-runtime-l1-1-0.dll
 0001:00001c74       _initterm_e                0000000180002c74 f   ucrt:api-ms-win-crt-runtime-l1-1-0.dll
 0001:00001c7a       _seh_filter_dll            0000000180002c7a f   ucrt:api-ms-win-crt-runtime-l1-1-0.dll
 0001:00001c80       _configure_narrow_argv     0000000180002c80 f   ucrt:api-ms-win-crt-runtime-l1-1-0.dll
 0001:00001c86       _initialize_narrow_environment 0000000180002c86 f   ucrt:api-ms-win-crt-runtime-l1-1-0.dll
 0001:00001c8c       _initialize_onexit_table   0000000180002c8c f   ucrt:api-ms-win-crt-runtime-l1-1-0.dll
 0001:00001c92       _register_onexit_function  0000000180002c92 f   ucrt:api-ms-win-crt-runtime-l1-1-0.dll
 0001:00001c98       _execute_onexit_table      0000000180002c98 f   ucrt:api-ms-win-crt-runtime-l1-1-0.dll
 0001:00001c9e       _crt_atexit                0000000180002c9e f   ucrt:api-ms-win-crt-runtime-l1-1-0.dll
 0001:00001ca4       _cexit                     0000000180002ca4 f   ucrt:api-ms-win-crt-runtime-l1-1-0.dll
 0001:00001cac       __acrt_initialize          0000000180002cac f   MSVCRT:ucrt_stubs.obj
 0001:00001cac       __acrt_thread_attach       0000000180002cac f   MSVCRT:ucrt_stubs.obj
 0001:00001cac       __acrt_thread_detach       0000000180002cac f   MSVCRT:ucrt_stubs.obj
 0001:00001cac       __acrt_uninitialize        0000000180002cac f   MSVCRT:ucrt_stubs.obj
 0001:00001cac       __acrt_uninitialize_critical 0000000180002cac f   MSVCRT:ucrt_stubs.obj
 0001:00001cac       __scrt_stub_for_acrt_initialize 0000000180002cac f   MSVCRT:ucrt_stubs.obj
 0001:00001cac       __scrt_stub_for_acrt_thread_attach 0000000180002cac f   MSVCRT:ucrt_stubs.obj
 0001:00001cac       __scrt_stub_for_acrt_thread_detach 0000000180002cac f   MSVCRT:ucrt_stubs.obj
 0001:00001cac       __scrt_stub_for_acrt_uninitialize 0000000180002cac f   MSVCRT:ucrt_stubs.obj
 0001:00001cac       __scrt_stub_for_acrt_uninitialize_critical 0000000180002cac f   MSVCRT:ucrt_stubs.obj
 0001:00001cac       __vcrt_initialize          0000000180002cac f   MSVCRT:ucrt_stubs.obj
 0001:00001cac       __vcrt_thread_attach       0000000180002cac f   MSVCRT:ucrt_stubs.obj
 0001:00001cac       __vcrt_thread_detach       0000000180002cac f   MSVCRT:ucrt_stubs.obj
 0001:00001cac       __vcrt_uninitialize        0000000180002cac f   MSVCRT:ucrt_stubs.obj
 0001:00001cac       __vcrt_uninitialize_critical 0000000180002cac f   MSVCRT:ucrt_stubs.obj
 0001:00001cb0       __scrt_stub_for_is_c_termination_complete 0000000180002cb0 f   MSVCRT:ucrt_stubs.obj
 0001:00001cb0       _is_c_termination_complete 0000000180002cb0 f   MSVCRT:ucrt_stubs.obj
 0001:00001cb3       memcpy                     0000000180002cb3 f   vcruntime:VCRUNTIME140.dll
 0001:00001cd0       _guard_dispatch_icall_nop  0000000180002cd0 f   MSVCRT:guard_dispatch.obj
 0001:00001cf0       _guard_xfg_dispatch_icall_nop 0000000180002cf0 f   MSVCRT:guard_xfg_dispatch.obj
 0002:00000000       __imp_CloseHandle          0000000180003000     kernel32:KERNEL32.dll
 0002:00000008       __imp_EnterCriticalSection 0000000180003008     kernel32:KERNEL32.dll
 0002:00000010       __imp_LeaveCriticalSection 0000000180003010     kernel32:KERNEL32.dll
 0002:00000018       __imp_InitializeCriticalSectionAndSpinCount 0000000180003018     kernel32:KERNEL32.dll
 0002:00000020       __imp_DeleteCriticalSection 0000000180003020     kernel32:KERNEL32.dll
 0002:00000028       __imp_SetEvent             0000000180003028     kernel32:KERNEL32.dll
 0002:00000030       __imp_ResetEvent           0000000180003030     kernel32:KERNEL32.dll
 0002:00000038       __imp_WaitForSingleObjectEx 0000000180003038     kernel32:KERNEL32.dll
 0002:00000040       __imp_CreateEventW         0000000180003040     kernel32:KERNEL32.dll
 0002:00000048       __imp_GetModuleHandleW     0000000180003048     kernel32:KERNEL32.dll
 0002:00000050       __imp_GetProcAddress       0000000180003050     kernel32:KERNEL32.dll
 0002:00000058       __imp_RtlCaptureContext    0000000180003058     kernel32:KERNEL32.dll
 0002:00000060       __imp_RtlLookupFunctionEntry 0000000180003060     kernel32:KERNEL32.dll
 0002:00000068       __imp_RtlVirtualUnwind     0000000180003068     kernel32:KERNEL32.dll
 0002:00000070       __imp_IsDebuggerPresent    0000000180003070     kernel32:KERNEL32.dll
 0002:00000078       __imp_UnhandledExceptionFilter 0000000180003078     kernel32:KERNEL32.dll
 0002:00000080       __imp_SetUnhandledExceptionFilter 0000000180003080     kernel32:KERNEL32.dll
 0002:00000088       __imp_IsProcessorFeaturePresent 0000000180003088     kernel32:KERNEL32.dll
 0002:00000090       __imp_GetCurrentProcess    0000000180003090     kernel32:KERNEL32.dll
 0002:00000098       __imp_TerminateProcess     0000000180003098     kernel32:KERNEL32.dll
 0002:000000a0       __imp_QueryPerformanceCounter 00000001800030a0     kernel32:KERNEL32.dll
 0002:000000a8       __imp_GetCurrentProcessId  00000001800030a8     kernel32:KERNEL32.dll
 0002:000000b0       __imp_GetCurrentThreadId   00000001800030b0     kernel32:KERNEL32.dll
 0002:000000b8       __imp_GetSystemTimeAsFileTime 00000001800030b8     kernel32:KERNEL32.dll
 0002:000000c0       __imp_DisableThreadLibraryCalls 00000001800030c0     kernel32:KERNEL32.dll
 0002:000000c8       __imp_InitializeSListHead  00000001800030c8     kernel32:KERNEL32.dll
 0002:000000d0       \177KERNEL32_NULL_THUNK_DATA 00000001800030d0     kernel32:KERNEL32.dll
 0002:000000d8       __imp_memset               00000001800030d8     vcruntime:VCRUNTIME140.dll
 0002:000000e0       __imp___C_specific_handler 00000001800030e0     vcruntime:VCRUNTIME140.dll
 0002:000000e8       __imp___std_type_info_destroy_list 00000001800030e8     vcruntime:VCRUNTIME140.dll
 0002:000000f0       __imp_memcpy               00000001800030f0     vcruntime:VCRUNTIME140.dll
 0002:000000f8       \177VCRUNTIME140_NULL_THUNK_DATA 00000001800030f8     vcruntime:VCRUNTIME140.dll
 0002:00000100       __imp__initialize_narrow_environment 0000000180003100     ucrt:api-ms-win-crt-runtime-l1-1-0.dll
 0002:00000108       __imp__cexit               0000000180003108     ucrt:api-ms-win-crt-runtime-l1-1-0.dll
 0002:00000110       __imp__crt_atexit          0000000180003110     ucrt:api-ms-win-crt-runtime-l1-1-0.dll
 0002:00000118       __imp__execute_onexit_table 0000000180003118     ucrt:api-ms-win-crt-runtime-l1-1-0.dll
 0002:00000120       __imp__register_onexit_function 0000000180003120     ucrt:api-ms-win-crt-runtime-l1-1-0.dll
 0002:00000128       __imp__initterm            0000000180003128     ucrt:api-ms-win-crt-runtime-l1-1-0.dll
 0002:00000130       __imp__initterm_e          0000000180003130     ucrt:api-ms-win-crt-runtime-l1-1-0.dll
 0002:00000138       __imp__seh_filter_dll      0000000180003138     ucrt:api-ms-win-crt-runtime-l1-1-0.dll
 0002:00000140       __imp__initialize_onexit_table 0000000180003140     ucrt:api-ms-win-crt-runtime-l1-1-0.dll
 0002:00000148       __imp__configure_narrow_argv 0000000180003148     ucrt:api-ms-win-crt-runtime-l1-1-0.dll
 0002:00000150       \177api-ms-win-crt-runtime-l1-1-0_NULL_THUNK_DATA 0000000180003150     ucrt:api-ms-win-crt-runtime-l1-1-0.dll
 0002:00000158       __imp___acrt_iob_func      0000000180003158     ucrt:api-ms-win-crt-stdio-l1-1-0.dll
 0002:00000160       __imp___stdio_common_vfprintf 0000000180003160     ucrt:api-ms-win-crt-stdio-l1-1-0.dll
 0002:00000168       __imp_fflush               0000000180003168     ucrt:api-ms-win-crt-stdio-l1-1-0.dll
 0002:00000170       \177api-ms-win-crt-stdio-l1-1-0_NULL_THUNK_DATA 0000000180003170     ucrt:api-ms-win-crt-stdio-l1-1-0.dll
 0002:00000178       __imp_strlen               0000000180003178     ucrt:api-ms-win-crt-string-l1-1-0.dll
 0002:00000180       __imp_strncpy              0000000180003180     ucrt:api-ms-win-crt-string-l1-1-0.dll
 0002:00000188       __imp_strcmp               0000000180003188     ucrt:api-ms-win-crt-string-l1-1-0.dll
 0002:00000190       \177api-ms-win-crt-string-l1-1-0_NULL_THUNK_DATA 0000000180003190     ucrt:api-ms-win-crt-string-l1-1-0.dll
 0002:00000198       __guard_check_icall_fptr   0000000180003198     MSVCRT:guard_support.obj
 0002:000001a0       __guard_xfg_check_icall_fptr 00000001800031a0     MSVCRT:guard_support.obj
 0002:000001a8       __guard_dispatch_icall_fptr 00000001800031a8     MSVCRT:guard_support.obj
 0002:000001b0       __guard_xfg_dispatch_icall_fptr 00000001800031b0     MSVCRT:guard_support.obj
 0002:000001b8       __guard_xfg_table_dispatch_icall_fptr 00000001800031b8     MSVCRT:guard_support.obj
 0002:000001c0       __castguard_check_failure_os_handled_fptr 00000001800031c0     MSVCRT:guard_support.obj
 0002:000001c8       __guard_memcpy_fptr        00000001800031c8     vcruntime:softmemtag.obj
 0002:000001d0       __xc_a                     00000001800031d0     MSVCRT:initializers.obj
 0002:000001d8       __xc_z                     00000001800031d8     MSVCRT:initializers.obj
 0002:000001e0       __xi_a                     00000001800031e0     MSVCRT:initializers.obj
 0002:000001f0       __xi_z                     00000001800031f0     MSVCRT:initializers.obj
 0002:000001f8       __xl_a                     00000001800031f8     MSVCRT:tlssup.obj
 0002:00000200       __xl_z                     0000000180003200     MSVCRT:tlssup.obj
 0002:00000208       __xp_a                     0000000180003208     MSVCRT:initializers.obj
 0002:00000210       __xp_z                     0000000180003210     MSVCRT:initializers.obj
 0002:00000218       __xt_a                     0000000180003218     MSVCRT:initializers.obj
 0002:00000220       __xt_z                     0000000180003220     MSVCRT:initializers.obj
 0002:00000268       ??_C@_0DM@KLJPMIDM@check_jvmti_status?3?5JVMTI?5funct@ 0000000180003268     liballthr01.obj
 0002:000002a8       ??_C@_0CA@CCEFGCFD@Fatal?5Error?5in?5RawMonitorEnter?4@ 00000001800032a8     liballthr01.obj
 0002:000002c8       ??_C@_0BP@POHFIHGF@Fatal?5Error?5in?5RawMonitorWait?4@ 00000001800032c8     liballthr01.obj
 0002:000002e8       ??_C@_0CB@HBCCEOBO@Fatal?5Error?5in?5RawMonitorNotify@ 00000001800032e8     liballthr01.obj
 0002:00000310       ??_C@_0CL@MEELKAEL@deallocate?3?5error?5in?5JVMTI?5Deal@ 0000000180003310     liballthr01.obj
 0002:00000340       ??_C@_0CP@IBPBEBM@get_method_class_name?3?5error?5in@ 0000000180003340     liballthr01.obj
 0002:00000370       ??_C@_01EEMJAFIK@?6@       0000000180003370     liballthr01.obj
 0002:00000378       ??_C@_0BB@NEONAMMP@?$DMUnnamed?5thread?$DO@ 0000000180003378     liballthr01.obj
 0002:00000390       ??_C@_0DD@PEIMAGBL@get_thread_name?3?5error?5in?5JVMTI@ 0000000180003390     liballthr01.obj
 0002:000003c8       ??_C@_0BB@JCNMKLLK@JVMTI_ERROR_NONE@ 00000001800033c8     liballthr01.obj
 0002:000003e0       ??_C@_0BL@LDIMKLPH@JVMTI_ERROR_INVALID_THREAD@ 00000001800033e0     liballthr01.obj
 0002:00000400       ??_C@_0CB@PJFPAIKJ@JVMTI_ERROR_INVALID_THREAD_GROU@ 0000000180003400     liballthr01.obj
 0002:00000428       ??_C@_0BN@LLMKHMNF@JVMTI_ERROR_INVALID_PRIORITY@ 0000000180003428     liballthr01.obj
 0002:00000448       ??_C@_0CB@MBOFKAGB@JVMTI_ERROR_THREAD_NOT_SUSPENDE@ 0000000180003448     liballthr01.obj
 0002:00000470       ??_C@_0BN@FABOLPBI@JVMTI_ERROR_THREAD_SUSPENDED@ 0000000180003470     liballthr01.obj
 0002:00000490       ??_C@_0BN@FDGNOBJM@JVMTI_ERROR_THREAD_NOT_ALIVE@ 0000000180003490     liballthr01.obj
 0002:000004b0       ??_C@_0BL@GOBIFKNJ@JVMTI_ERROR_INVALID_OBJECT@ 00000001800034b0     liballthr01.obj
 0002:000004d0       ??_C@_0BK@FCMAJPPC@JVMTI_ERROR_INVALID_CLASS@ 00000001800034d0     liballthr01.obj
 0002:000004f0       ??_C@_0BP@IKLLBKEB@JVMTI_ERROR_CLASS_NOT_PREPARED@ 00000001800034f0     liballthr01.obj
 0002:00000510       ??_C@_0BN@KLPPLKG@JVMTI_ERROR_INVALID_METHODID@ 0000000180003510     liballthr01.obj
 0002:00000530       ??_C@_0BN@BCEKOKND@JVMTI_ERROR_INVALID_LOCATION@ 0000000180003530     liballthr01.obj
 0002:00000550       ??_C@_0BM@DFDGPME@JVMTI_ERROR_INVALID_FIELDID@ 0000000180003550     liballthr01.obj
 0002:00000570       ??_C@_0BL@NELIEPEC@JVMTI_ERROR_NO_MORE_FRAMES@ 0000000180003570     liballthr01.obj
 0002:00000590       ??_C@_0BJ@BDBECFDM@JVMTI_ERROR_OPAQUE_FRAME@ 0000000180003590     liballthr01.obj
 0002:000005b0       ??_C@_0BK@MIIFNLOB@JVMTI_ERROR_TYPE_MISMATCH@ 00000001800035b0     liballthr01.obj
 0002:000005d0       ??_C@_0BJ@HPCAOILC@JVMTI_ERROR_INVALID_SLOT@ 00000001800035d0     liballthr01.obj
 0002:000005f0       ??_C@_0BG@CHILOPNI@JVMTI_ERROR_DUPLICATE@ 00000001800035f0     liballthr01.obj
 0002:00000608       ??_C@_0BG@DIEMLHKM@JVMTI_ERROR_NOT_FOUND@ 0000000180003608     liballthr01.obj
 0002:00000620       ??_C@_0BM@NHMCKHOB@JVMTI_ERROR_INVALID_MONITOR@ 0000000180003620     liballthr01.obj
 0002:00000640       ??_C@_0BO@PPEDAJGL@JVMTI_ERROR_NOT_MONITOR_OWNER@ 0000000180003640     liballthr01.obj
 0002:00000660       ??_C@_0BG@FCAIPEID@JVMTI_ERROR_INTERRUPT@ 0000000180003660     liballthr01.obj
 0002:00000678       ??_C@_0CB@EGDBNKOI@JVMTI_ERROR_INVALID_CLASS_FORMA@ 0000000180003678     liballthr01.obj
 0002:000006a0       ??_C@_0CG@DGKOGIAL@JVMTI_ERROR_CIRCULAR_CLASS_DEFI@ 00000001800036a0     liballthr01.obj
 0002:000006c8       ??_C@_0BP@ICEALPKC@JVMTI_ERROR_FAILS_VERIFICATION@ 00000001800036c8     liballthr01.obj
 0002:000006e8       ??_C@_0DC@JDACLMIO@JVMTI_ERROR_UNSUPPORTED_REDEFIN@ 00000001800036e8     liballthr01.obj
 0002:00000720       ??_C@_0DE@GKDKNOMJ@JVMTI_ERROR_UNSUPPORTED_REDEFIN@ 0000000180003720     liballthr01.obj
 0002:00000758       ??_C@_0BO@LAFKIOG@JVMTI_ERROR_INVALID_TYPESTATE@ 0000000180003758     liballthr01.obj
 0002:00000778       ??_C@_0DH@INDGCLLB@JVMTI_ERROR_UNSUPPORTED_REDEFIN@ 0000000180003778     liballthr01.obj
 0002:000007b0       ??_C@_0DE@NHEOMMGI@JVMTI_ERROR_UNSUPPORTED_REDEFIN@ 00000001800037b0     liballthr01.obj
 0002:000007e8       ??_C@_0CA@EKPNJOEP@JVMTI_ERROR_UNSUPPORTED_VERSION@ 00000001800037e8     liballthr01.obj
 0002:00000808       ??_C@_0BN@OFFMAHHL@JVMTI_ERROR_NAMES_DONT_MATCH@ 0000000180003808     liballthr01.obj
 0002:00000828       ??_C@_0DN@HHBBLAKE@JVMTI_ERROR_UNSUPPORTED_REDEFIN@ 0000000180003828     liballthr01.obj
 0002:00000868       ??_C@_0DO@HMBGBGNA@JVMTI_ERROR_UNSUPPORTED_REDEFIN@ 0000000180003868     liballthr01.obj
 0002:000008a8       ??_C@_0BP@PBECGKHJ@JVMTI_ERROR_UNMODIFIABLE_CLASS@ 00000001800038a8     liballthr01.obj
 0002:000008c8       ??_C@_0BK@CANILEHF@JVMTI_ERROR_NOT_AVAILABLE@ 00000001800038c8     liballthr01.obj
 0002:000008e8       ??_C@_0CE@INJKMEFK@JVMTI_ERROR_MUST_POSSESS_CAPABI@ 00000001800038e8     liballthr01.obj
 0002:00000910       ??_C@_0BJ@LBFPFPDM@JVMTI_ERROR_NULL_POINTER@ 0000000180003910     liballthr01.obj
 0002:00000930       ??_C@_0BP@CHJPNNEM@JVMTI_ERROR_ABSENT_INFORMATION@ 0000000180003930     liballthr01.obj
 0002:00000950       ??_C@_0BP@OMFMNLC@JVMTI_ERROR_INVALID_EVENT_TYPE@ 0000000180003950     liballthr01.obj
 0002:00000970       ??_C@_0BN@BIBNPHHO@JVMTI_ERROR_ILLEGAL_ARGUMENT@ 0000000180003970     liballthr01.obj
 0002:00000990       ??_C@_0BK@KKNDHDCE@JVMTI_ERROR_NATIVE_METHOD@ 0000000180003990     liballthr01.obj
 0002:000009b0       ??_C@_0BK@PMKCFHAE@JVMTI_ERROR_OUT_OF_MEMORY@ 00000001800039b0     liballthr01.obj
 0002:000009d0       ??_C@_0BK@NNJBDMNB@JVMTI_ERROR_ACCESS_DENIED@ 00000001800039d0     liballthr01.obj
 0002:000009f0       ??_C@_0BI@GHECLMNC@JVMTI_ERROR_WRONG_PHASE@ 00000001800039f0     liballthr01.obj
 0002:00000a08       ??_C@_0BF@OLIHJOII@JVMTI_ERROR_INTERNAL@ 0000000180003a08     liballthr01.obj
 0002:00000a20       ??_C@_0BO@EOHGKJHI@JVMTI_ERROR_UNATTACHED_THREAD@ 0000000180003a20     liballthr01.obj
 0002:00000a40       ??_C@_0CA@LKHFDACL@JVMTI_ERROR_INVALID_ENVIRONMENT@ 0000000180003a40     liballthr01.obj
 0002:00000a60       ??_C@_0BA@MMFHLOKK@?$DMunknown?5error?$DO@ 0000000180003a60     liballthr01.obj
 0002:00000a70       ??_C@_0BB@NOKBFPFO@java?1lang?1Thread@ 0000000180003a70     liballthr01.obj
 0002:00000a88       ??_C@_0BG@IKDDPPGD@?$CILjava?1lang?1String?$DL?$CJV@ 0000000180003a88     liballthr01.obj
 0002:00000aa0       ??_C@_06FALKBLGB@?$DMinit?$DO@ 0000000180003aa0     liballthr01.obj
 0002:00000aa8       ??_C@_0CJ@KCDEKOCJ@Wrong?5result?5of?5a?5valid?5call?5to@ 0000000180003aa8     liballthr01.obj
 0002:00000ad8       ??_C@_0CN@LKPEOJPO@?$CIAddCapabilities?$CJ?5unexpected?5er@ 0000000180003ad8     liballthr01.obj
 0002:00000b08       ??_C@_0BL@LBNAKAK@_started_agent_thread_lock@ 0000000180003b08     liballthr01.obj
 0002:00000b28       ??_C@_0BM@NBCJKEJP@_stopping_agent_thread_lock@ 0000000180003b28     liballthr01.obj
 0002:00000b48       ??_C@_0BG@EOKANEHL@?5?$DO?$DO?$DO?5Check?5point?3?5?$CFd?6@ 0000000180003b48     liballthr01.obj
 0002:00000b60       ??_C@_0BI@HGJHMBJL@Failed?5in?5GetAllThreads@ 0000000180003b60     liballthr01.obj
 0002:00000b78       ??_C@_0BI@HEAODMFN@Failed?5in?5GetThreadInfo@ 0000000180003b78     liballthr01.obj
 0002:00000b90       ??_C@_07CBDAPNPF@?5?$DO?$DO?$DO?5?$CFs@ 0000000180003b90     liballthr01.obj
 0002:00000b98       ??_C@_0CJ@KHBKLDNE@Point?5?$CFd?3?5detected?5unexpected?5t@ 0000000180003b98     liballthr01.obj
 0002:00000bc8       ??_C@_0CC@HBDBKALG@Point?5?$CFd?3?5thread?5?$CFs?5not?5detecte@ 0000000180003bc8     liballthr01.obj
 0002:00000bf0       ??_C@_0BK@HBJIHGIA@Failed?5to?5run?5AgentThread@ 0000000180003bf0     liballthr01.obj
 0002:00000c10       ??_C@_0BG@HJJEOENG@Started?5Agent?5Thread?6@ 0000000180003c10     liballthr01.obj
 0002:00000c28       ??_C@_0BG@BPHAHOEG@Stopped?5Agent?5Thread?6@ 0000000180003c28     liballthr01.obj
 0002:00000c40       ??_C@_1EC@JIJBPKFM@?$AAa?$AAp?$AAi?$AA?9?$AAm?$AAs?$AA?9?$AAw?$AAi?$AAn?$AA?9?$AAc?$AAo?$AAr?$AAe@ 0000000180003c40     MSVCRT:thread_safe_statics.obj
 0002:00000c88       ??_C@_1BK@MGMFAEKH@?$AAk?$AAe?$AAr?$AAn?$AAe?$AAl?$AA3?$AA2?$AA?4?$AAd?$AAl?$AAl@ 0000000180003c88     MSVCRT:thread_safe_statics.obj
 0002:00000ca8       ??_C@_0BJ@JEBJOJFJ@SleepConditionVariableCS@ 0000000180003ca8     MSVCRT:thread_safe_statics.obj
 0002:00000cc8       ??_C@_0BJ@PGPPEPCC@WakeAllConditionVariable@ 0000000180003cc8     MSVCRT:thread_safe_statics.obj
 0002:00000ce8       _pDefaultRawDllMain        0000000180003ce8     MSVCRT:dll_dllmain.obj
 0002:00000ce8       _pRawDllMain               0000000180003ce8     MSVCRT:dll_dllmain.obj
 0002:00000cf0       __xmm@ffffffffffffffffffffffffffffffff 0000000180003cf0     MSVCRT:utility.obj
 0002:00000d10       _load_config_used          0000000180003d10     MSVCRT:loadcfg.obj
 0002:00000f00       _tls_used                  0000000180003f00     MSVCRT:tlssup.obj
 0002:00000f28       __volatile_metadata        0000000180003f28     <linker-defined>
 0002:000012a8       __rtc_iaa                  00000001800042a8     MSVCRT:initsect.obj
 0002:000012b0       __rtc_izz                  00000001800042b0     MSVCRT:initsect.obj
 0002:000012b8       __rtc_taa                  00000001800042b8     MSVCRT:initsect.obj
 0002:000012c0       __rtc_tzz                  00000001800042c0     MSVCRT:initsect.obj
 0002:000012c8       _tls_start                 00000001800042c8     MSVCRT:tlssup.obj
 0002:000012cc       _Init_thread_epoch         00000001800042cc     MSVCRT:thread_safe_statics.obj
 0002:000012d0       _tls_end                   00000001800042d0     MSVCRT:tlssup.obj
 0002:000015c8       __IMPORT_DESCRIPTOR_KERNEL32 00000001800045c8     kernel32:KERNEL32.dll
 0002:000015dc       __IMPORT_DESCRIPTOR_VCRUNTIME140 00000001800045dc     vcruntime:VCRUNTIME140.dll
 0002:000015f0       __IMPORT_DESCRIPTOR_api-ms-win-crt-stdio-l1-1-0 00000001800045f0     ucrt:api-ms-win-crt-stdio-l1-1-0.dll
 0002:00001604       __IMPORT_DESCRIPTOR_api-ms-win-crt-string-l1-1-0 0000000180004604     ucrt:api-ms-win-crt-string-l1-1-0.dll
 0002:00001618       __IMPORT_DESCRIPTOR_api-ms-win-crt-runtime-l1-1-0 0000000180004618     ucrt:api-ms-win-crt-runtime-l1-1-0.dll
 0002:0000162c       __NULL_IMPORT_DESCRIPTOR   000000018000462c     kernel32:KERNEL32.dll
 0003:00000128       _Init_global_epoch         0000000180005128     MSVCRT:thread_safe_statics.obj
 0003:00000130       __security_cookie          0000000180005130     MSVCRT:gs_cookie.obj
 0003:00000138       __security_cookie_complement 0000000180005138     MSVCRT:gs_cookie.obj
 0003:00000140       __scrt_native_dllmain_reason 0000000180005140     MSVCRT:utility.obj
 0003:00000148       __isa_available            0000000180005148     MSVCRT:cpu_disp.obj
 0003:0000014c       __isa_enabled              000000018000514c     MSVCRT:cpu_disp.obj
 0003:00000150       __memset_fast_string_threshold 0000000180005150     MSVCRT:cpu_disp.obj
 0003:00000158       __memset_nt_threshold      0000000180005158     MSVCRT:cpu_disp.obj
 0003:00000160       __scrt_ucrt_dll_is_in_use  0000000180005160     MSVCRT:ucrt_stubs.obj
 0003:00000170       ?_OptionsStorage@?1??__local_stdio_printf_options@@9@4_KA 0000000180005170     liballthr01.obj
 0003:000001e8       _tls_index                 00000001800051e8     MSVCRT:tlssup.obj
 0003:000001f0       __scrt_current_native_startup_state 00000001800051f0     MSVCRT:utility.obj
 0003:000001f8       __scrt_native_startup_lock 00000001800051f8     MSVCRT:utility.obj
 0003:00000238       __scrt_debugger_hook_flag  0000000180005238     MSVCRT:utility_desktop.obj
 0003:000007b0       ?__type_info_root_node@@3U__type_info_node@@A 00000001800057b0     MSVCRT:tncleanup.obj
 0003:000007c0       ?_OptionsStorage@?1??__local_stdio_scanf_options@@9@4_KA 00000001800057c0     MSVCRT:default_local_stdio_options.obj
 0003:000007c8       __favor                    00000001800057c8     MSVCRT:cpu_disp.obj
 0003:000007d0       __dyn_tls_init_callback    00000001800057d0     <common>

 entry point at        0001:00001260

 Static symbols

 0000:ffff8000       .debug$S                   0000000180000000     allthr01.exp
 0000:ffff8000       .debug$S                   0000000180000000     vcruntime:VCRUNTIME140.dll
 0000:ffff8000       .debug$S                   0000000180000000     vcruntime:VCRUNTIME140.dll
 0000:ffff8000       .debug$S                   0000000180000000     vcruntime:VCRUNTIME140.dll
 0000:ffff8000       .debug$S                   0000000180000000     vcruntime:VCRUNTIME140.dll
 0000:ffff8000       .debug$S                   0000000180000000     vcruntime:VCRUNTIME140.dll
 0000:ffff8000       .debug$S                   0000000180000000     vcruntime:VCRUNTIME140.dll
 0000:ffff8000       .debug$S                   0000000180000000     ucrt:api-ms-win-crt-runtime-l1-1-0.dll
 0000:ffff8000       .debug$S                   0000000180000000     ucrt:api-ms-win-crt-runtime-l1-1-0.dll
 0000:ffff8000       .debug$S                   0000000180000000     ucrt:api-ms-win-crt-runtime-l1-1-0.dll
 0000:ffff8000       .debug$S                   0000000180000000     ucrt:api-ms-win-crt-runtime-l1-1-0.dll
 0000:ffff8000       .debug$S                   0000000180000000     ucrt:api-ms-win-crt-runtime-l1-1-0.dll
 0000:ffff8000       .debug$S                   0000000180000000     ucrt:api-ms-win-crt-runtime-l1-1-0.dll
 0000:ffff8000       .debug$S                   0000000180000000     ucrt:api-ms-win-crt-runtime-l1-1-0.dll
 0000:ffff8000       .debug$S                   0000000180000000     ucrt:api-ms-win-crt-runtime-l1-1-0.dll
 0000:ffff8000       .debug$S                   0000000180000000     ucrt:api-ms-win-crt-runtime-l1-1-0.dll
 0000:ffff8000       .debug$S                   0000000180000000     ucrt:api-ms-win-crt-runtime-l1-1-0.dll
 0000:ffff8000       .debug$S                   0000000180000000     ucrt:api-ms-win-crt-runtime-l1-1-0.dll
 0000:ffff8000       .debug$S                   0000000180000000     ucrt:api-ms-win-crt-runtime-l1-1-0.dll
 0000:ffff8000       .debug$S                   0000000180000000     ucrt:api-ms-win-crt-stdio-l1-1-0.dll
 0000:ffff8000       .debug$S                   0000000180000000     ucrt:api-ms-win-crt-stdio-l1-1-0.dll
 0000:ffff8000       .debug$S                   0000000180000000     ucrt:api-ms-win-crt-stdio-l1-1-0.dll
 0000:ffff8000       .debug$S                   0000000180000000     ucrt:api-ms-win-crt-string-l1-1-0.dll
 0000:ffff8000       .debug$S                   0000000180000000     ucrt:api-ms-win-crt-string-l1-1-0.dll
 0000:ffff8000       .debug$S                   0000000180000000     ucrt:api-ms-win-crt-string-l1-1-0.dll
 0000:ffff8000       .debug$S                   0000000180000000     ucrt:api-ms-win-crt-string-l1-1-0.dll
 0000:ffff8000       .debug$S                   0000000180000000     ucrt:api-ms-win-crt-string-l1-1-0.dll
 0000:ffff8000       .debug$S                   0000000180000000     kernel32:KERNEL32.dll
 0000:ffff8000       .debug$S                   0000000180000000     kernel32:KERNEL32.dll
 0000:ffff8000       .debug$S                   0000000180000000     kernel32:KERNEL32.dll
 0000:ffff8000       .debug$S                   0000000180000000     kernel32:KERNEL32.dll
 0000:ffff8000       .debug$S                   0000000180000000     kernel32:KERNEL32.dll
 0000:ffff8000       .debug$S                   0000000180000000     kernel32:KERNEL32.dll
 0000:ffff8000       .debug$S                   0000000180000000     kernel32:KERNEL32.dll
 0000:ffff8000       .debug$S                   0000000180000000     kernel32:KERNEL32.dll
 0000:ffff8000       .debug$S                   0000000180000000     kernel32:KERNEL32.dll
 0000:ffff8000       .debug$S                   0000000180000000     kernel32:KERNEL32.dll
 0000:ffff8000       .debug$S                   0000000180000000     kernel32:KERNEL32.dll
 0000:ffff8000       .debug$S                   0000000180000000     kernel32:KERNEL32.dll
 0000:ffff8000       .debug$S                   0000000180000000     kernel32:KERNEL32.dll
 0000:ffff8000       .debug$S                   0000000180000000     kernel32:KERNEL32.dll
 0000:ffff8000       .debug$S                   0000000180000000     kernel32:KERNEL32.dll
 0000:ffff8000       .debug$S                   0000000180000000     kernel32:KERNEL32.dll
 0000:ffff8000       .debug$S                   0000000180000000     kernel32:KERNEL32.dll
 0000:ffff8000       .debug$S                   0000000180000000     kernel32:KERNEL32.dll
 0000:ffff8000       .debug$S                   0000000180000000     kernel32:KERNEL32.dll
 0000:ffff8000       .debug$S                   0000000180000000     kernel32:KERNEL32.dll
 0000:ffff8000       .debug$S                   0000000180000000     kernel32:KERNEL32.dll
 0000:ffff8000       .debug$S                   0000000180000000     kernel32:KERNEL32.dll
 0000:ffff8000       .debug$S                   0000000180000000     kernel32:KERNEL32.dll
 0000:ffff8000       .debug$S                   0000000180000000     kernel32:KERNEL32.dll
 0000:ffff8000       .debug$S                   0000000180000000     kernel32:KERNEL32.dll
 0000:ffff8000       .debug$S                   0000000180000000     kernel32:KERNEL32.dll
 0000:ffff8000       .debug$S                   0000000180000000     kernel32:KERNEL32.dll
 0000:ffff8000       .debug$S                   0000000180000000     kernel32:KERNEL32.dll
 0001:000002e0       ?check_jvmti_status@@YAXPEAUJNIEnv_@@W4jvmtiError@@PEBD@Z 00000001800012e0 f   liballthr01.obj
 0001:00000374       ?get_thread_name@@YAPEADPEAU_jvmtiEnv@@PEAUJNIEnv_@@PEAV_jobject@@@Z 0000000180001374 f   liballthr01.obj
 0001:00000b10       sys_thread                 0000000180001b10 f   liballthr01.obj
 0001:00000c24       ?__scrt_initialize_thread_safe_statics@@YAHXZ 0000000180001c24 f   MSVCRT:thread_safe_statics.obj
 0001:00000cf4       ?__scrt_uninitialize_thread_safe_statics@@YAXXZ 0000000180001cf4 f   MSVCRT:thread_safe_statics.obj
 0001:00000f10       $$000000                   0000000180001f10     MSVCRT:amdsecgs.obj
 0001:00000f40       ?dllmain_crt_dispatch@@YAHQEAUHINSTANCE__@@KQEAX@Z 0000000180001f40 f   MSVCRT:dll_dllmain.obj
 0001:00000f90       ?dllmain_crt_process_attach@@YAHQEAUHINSTANCE__@@QEAX@Z 0000000180001f90 f   MSVCRT:dll_dllmain.obj
 0001:000010a8       ?dllmain_crt_process_detach@@YAH_N@Z 00000001800020a8 f   MSVCRT:dll_dllmain.obj
 0001:0000112c       ?dllmain_dispatch@@YAHQEAUHINSTANCE__@@KQEAX@Z 000000018000212c f   MSVCRT:dll_dllmain.obj
 0001:00001880       capture_previous_context   0000000180002880 f   MSVCRT:gs_report.obj
 0001:00001cc0       $$000000                   0000000180002cc0     MSVCRT:guard_dispatch.obj
 0001:00001ce0       $$000000                   0000000180002ce0     MSVCRT:guard_xfg_dispatch.obj
 0001:00001cf6       ?fin$0@?0??dllmain_crt_process_attach@@YAHQEAUHINSTANCE__@@QEAX@Z@4HA 0000000180002cf6 f   MSVCRT:dll_dllmain.obj
 0001:00001d0d       ?fin$0@?0??dllmain_crt_process_detach@@YAH_N@Z@4HA 0000000180002d0d f   MSVCRT:dll_dllmain.obj
 0001:00001d26       ?fin$1@?0??dllmain_crt_process_detach@@YAH_N@Z@4HA 0000000180002d26 f   MSVCRT:dll_dllmain.obj
 0001:00001d3a       ?filt$0@?0??dllmain_dispatch@@YAHQEAUHINSTANCE__@@KQEAX@Z@4HA 0000000180002d3a f   MSVCRT:dll_dllmain.obj
 0001:00001d70       __scrt_is_nonwritable_in_current_image$filt$0 0000000180002d70 f   MSVCRT:utility.obj
 0002:000001e8       ?__scrt_initialize_tss_var@@3P6AHXZEA 00000001800031e8     MSVCRT:thread_safe_statics.obj
 0002:00000230       main_name                  0000000180003230     liballthr01.obj
 0002:00000238       thread1_name               0000000180003238     liballthr01.obj
 0002:00000240       sys_thread_name            0000000180003240     liballthr01.obj
 0002:00000250       fj_thread_name             0000000180003250     liballthr01.obj
 0002:00000d00       GS_ExceptionPointers       0000000180003d00     MSVCRT:gs_report.obj
 0002:000012d8       $unwind$printf             00000001800042d8     liballthr01.obj
 0002:000012e4       $unwind$?NewObject@JNIEnv_@@QEAAPEAV_jobject@@PEAV_jclass@@PEAU_jmethodID@@ZZ 00000001800042e4     liballthr01.obj
 0002:000012ec       $unwind$Agent_OnLoad       00000001800042ec     liballthr01.obj
 0002:000012fc       $unwind$?check_jvmti_status@@YAXPEAUJNIEnv_@@W4jvmtiError@@PEBD@Z 00000001800042fc     liballthr01.obj
 0002:0000130c       $unwind$?create_raw_monitor@@YAPEAU_jrawMonitorID@@PEAU_jvmtiEnv@@PEBD@Z 000000018000430c     liballthr01.obj
 0002:0000130c       $unwind$__scrt_initialize_default_local_stdio_options 000000018000430c     MSVCRT:default_local_stdio_options.obj
 0002:0000130c       $unwind$?dllmain_crt_dispatch@@YAHQEAUHINSTANCE__@@KQEAX@Z 000000018000430c     MSVCRT:dll_dllmain.obj
 0002:0000130c       $unwind$DllMain            000000018000430c     MSVCRT:dll_dllmain_stub.obj
 0002:0000130c       $unwind$__GSHandlerCheck   000000018000430c     MSVCRT:gshandler.obj
 0002:0000130c       $unwind$?__scrt_uninitialize_thread_safe_statics@@YAXXZ 000000018000430c     MSVCRT:thread_safe_statics.obj
 0002:0000130c       $unwind$_Init_thread_notify 000000018000430c     MSVCRT:thread_safe_statics.obj
 0002:0000130c       $unwind$__scrt_acquire_startup_lock 000000018000430c     MSVCRT:utility.obj
 0002:0000130c       $unwind$__scrt_dllmain_after_initialize_c 000000018000430c     MSVCRT:utility.obj
 0002:0000130c       $unwind$__scrt_dllmain_before_initialize_c 000000018000430c     MSVCRT:utility.obj
 0002:0000130c       $unwind$__scrt_dllmain_crt_thread_attach 000000018000430c     MSVCRT:utility.obj
 0002:0000130c       $unwind$__scrt_dllmain_crt_thread_detach 000000018000430c     MSVCRT:utility.obj
 0002:0000130c       $unwind$__scrt_dllmain_uninitialize_c 000000018000430c     MSVCRT:utility.obj
 0002:0000130c       $unwind$__scrt_dllmain_uninitialize_critical 000000018000430c     MSVCRT:utility.obj
 0002:0000130c       $unwind$atexit             000000018000430c     MSVCRT:utility.obj
 0002:00001314       $unwind$?get_thread_name@@YAPEADPEAU_jvmtiEnv@@PEAUJNIEnv_@@PEAV_jobject@@@Z 0000000180004314     liballthr01.obj
 0002:00001324       $unwind$create_jthread     0000000180004324     liballthr01.obj
 0002:00001338       $unwind$sys_thread         0000000180004338     liballthr01.obj
 0002:00001338       $unwind$__scrt_dllmain_exception_filter 0000000180004338     MSVCRT:utility.obj
 0002:0000134c       $unwind$check_info         000000018000434c     liballthr01.obj
 0002:00001364       $unwind$Java_allthr01_startAgentThread 0000000180004364     liballthr01.obj
 0002:00001374       $unwind$Java_allthr01_stopAgentThread 0000000180004374     liballthr01.obj
 0002:00001374       $unwind$_DllMainCRTStartup 0000000180004374     MSVCRT:dll_dllmain.obj
 0002:00001384       $unwind$__raise_securityfailure 0000000180004384     MSVCRT:gs_report.obj
 0002:00001384       $unwind$_Init_thread_footer 0000000180004384     MSVCRT:thread_safe_statics.obj
 0002:00001384       $unwind$_Init_thread_header 0000000180004384     MSVCRT:thread_safe_statics.obj
 0002:00001384       $unwind$_Init_thread_wait  0000000180004384     MSVCRT:thread_safe_statics.obj
 0002:00001384       $unwind$__scrt_initialize_crt 0000000180004384     MSVCRT:utility.obj
 0002:00001384       $unwind$__scrt_initialize_onexit_tables 0000000180004384     MSVCRT:utility.obj
 0002:00001384       $unwind$__scrt_release_startup_lock 0000000180004384     MSVCRT:utility.obj
 0002:00001384       $unwind$__scrt_uninitialize_crt 0000000180004384     MSVCRT:utility.obj
 0002:00001384       $unwind$_onexit            0000000180004384     MSVCRT:utility.obj
 0002:0000138c       $unwind$_RTC_Initialize    000000018000438c     MSVCRT:initsect.obj
 0002:0000138c       $unwind$_RTC_Terminate     000000018000438c     MSVCRT:initsect.obj
 0002:0000138c       $unwind$?__scrt_initialize_thread_safe_statics@@YAHXZ 000000018000438c     MSVCRT:thread_safe_statics.obj
 0002:00001398       $unwind$__GSHandlerCheckCommon 0000000180004398     MSVCRT:gshandler.obj
 0002:000013a0       $xdatasym                  00000001800043a0     MSVCRT:amdsecgs.obj
 0002:000013a4       $unwind$?dllmain_crt_process_attach@@YAHQEAUHINSTANCE__@@QEAX@Z 00000001800043a4     MSVCRT:dll_dllmain.obj
 0002:000013e0       $unwind$?fin$0@?0??dllmain_crt_process_attach@@YAHQEAUHINSTANCE__@@QEAX@Z@4HA 00000001800043e0     MSVCRT:dll_dllmain.obj
 0002:000013e0       $unwind$?fin$0@?0??dllmain_crt_process_detach@@YAH_N@Z@4HA 00000001800043e0     MSVCRT:dll_dllmain.obj
 0002:000013e0       $unwind$?fin$1@?0??dllmain_crt_process_detach@@YAH_N@Z@4HA 00000001800043e0     MSVCRT:dll_dllmain.obj
 0002:000013e8       $unwind$?dllmain_crt_process_detach@@YAH_N@Z 00000001800043e8     MSVCRT:dll_dllmain.obj
 0002:0000143c       $unwind$?dllmain_dispatch@@YAHQEAUHINSTANCE__@@KQEAX@Z 000000018000443c     MSVCRT:dll_dllmain.obj
 0002:00001464       $unwind$?filt$0@?0??dllmain_dispatch@@YAHQEAUHINSTANCE__@@KQEAX@Z@4HA 0000000180004464     MSVCRT:dll_dllmain.obj
 0002:0000146c       $unwind$__scrt_is_nonwritable_in_current_image 000000018000446c     MSVCRT:utility.obj
 0002:0000148c       $unwind$__scrt_is_nonwritable_in_current_image$filt$0 000000018000448c     MSVCRT:utility.obj
 0002:00001494       $unwind$__scrt_fastfail    0000000180004494     MSVCRT:utility_desktop.obj
 0002:000014a4       $unwind$__report_gsfailure 00000001800044a4     MSVCRT:gs_report.obj
 0002:000014ac       $unwind$capture_previous_context 00000001800044ac     MSVCRT:gs_report.obj
 0002:000014b8       $unwind$__security_init_cookie 00000001800044b8     MSVCRT:gs_support.obj
 0002:000014c4       $unwind$__isa_available_init 00000001800044c4     MSVCRT:cpu_disp.obj
 0002:000014d8       $xdatasym                  00000001800044d8     MSVCRT:guard_dispatch.obj
 0002:000014e0       $xdatasym                  00000001800044e0     MSVCRT:guard_xfg_dispatch.obj
 0002:000014f0       .edata                     00000001800044f0     allthr01.exp
 0002:00001518       rgpv                       0000000180004518     allthr01.exp
 0002:0000152c       rgszName                   000000018000452c     allthr01.exp
 0002:00001540       rgwOrd                     0000000180004540     allthr01.exp
 0002:0000154a       szName                     000000018000454a     allthr01.exp
 0002:00001557       $N00001                    0000000180004557     allthr01.exp
 0002:00001564       $N00002                    0000000180004564     allthr01.exp
 0002:0000157d       $N00003                    000000018000457d     allthr01.exp
 0002:0000159c       $N00004                    000000018000459c     allthr01.exp
 0002:000015ba       $N00005                    00000001800045ba     allthr01.exp
 0002:00001a24       .idata$6                   0000000180004a24     kernel32:KERNEL32.dll
 0002:00001a74       .idata$6                   0000000180004a74     vcruntime:VCRUNTIME140.dll
 0002:00001baa       .idata$6                   0000000180004baa     ucrt:api-ms-win-crt-stdio-l1-1-0.dll
 0002:00001bca       .idata$6                   0000000180004bca     ucrt:api-ms-win-crt-string-l1-1-0.dll
 0002:00001bec       .idata$6                   0000000180004bec     ucrt:api-ms-win-crt-runtime-l1-1-0.dll
 0003:00000000       main_only                  0000000180005000     liballthr01.obj
 0003:00000008       thr1_only                  0000000180005008     liballthr01.obj
 0003:00000010       sys_only                   0000000180005010     liballthr01.obj
 0003:00000018       main_thr1                  0000000180005018     liballthr01.obj
 0003:00000028       main_sys                   0000000180005028     liballthr01.obj
 0003:00000038       thr1_sys                   0000000180005038     liballthr01.obj
 0003:00000048       main_fj                    0000000180005048     liballthr01.obj
 0003:00000060       thr_info                   0000000180005060     liballthr01.obj
 0003:00000120       ?UNNAMED_STR@?1??get_thread_name@@YAPEADPEAU_jvmtiEnv@@PEAUJNIEnv_@@PEAV_jobject@@@Z@4PEBDEB 0000000180005120     liballthr01.obj
 0003:00000178       ?UNNAMED_LEN@?1??get_thread_name@@YAPEADPEAU_jvmtiEnv@@PEAUJNIEnv_@@PEAV_jobject@@@Z@4_KA 0000000180005178     liballthr01.obj
 0003:00000180       ?$TSS0@?1??get_thread_name@@YAPEADPEAU_jvmtiEnv@@PEAUJNIEnv_@@PEAV_jobject@@@Z@4HA 0000000180005180     liballthr01.obj
 0003:00000188       jvmti_env                  0000000180005188     liballthr01.obj
 0003:00000190       starting_agent_thread_lock 0000000180005190     liballthr01.obj
 0003:00000198       stopping_agent_thread_lock 0000000180005198     liballthr01.obj
 0003:000001a0       ?g_tss_cv@@3U_RTL_CONDITION_VARIABLE@@A 00000001800051a0     MSVCRT:thread_safe_statics.obj
 0003:000001a8       ?g_tss_event@@3PEAXEA      00000001800051a8     MSVCRT:thread_safe_statics.obj
 0003:000001b0       ?g_tss_mutex@@3U_RTL_CRITICAL_SECTION@@A 00000001800051b0     MSVCRT:thread_safe_statics.obj
 0003:000001d8       ?g_sleep_condition_variable_cs@@3P6AHPEAU_RTL_CONDITION_VARIABLE@@PEAU_RTL_CRITICAL_SECTION@@K@ZEA 00000001800051d8     MSVCRT:thread_safe_statics.obj
 0003:000001e0       ?g_wake_all_condition_variable@@3P6AXPEAU_RTL_CONDITION_VARIABLE@@@ZEA 00000001800051e0     MSVCRT:thread_safe_statics.obj
 0003:000001ec       ?__proc_attached@@3HA      00000001800051ec     MSVCRT:dll_dllmain.obj
 0003:00000200       ?is_initialized_as_dll@@3_NA 0000000180005200     MSVCRT:utility.obj
 0003:00000201       ?module_local_atexit_table_initialized@@3_NA 0000000180005201     MSVCRT:utility.obj
 0003:00000208       ?module_local_atexit_table@@3U_onexit_table_t@@A 0000000180005208     MSVCRT:utility.obj
 0003:00000220       ?module_local_at_quick_exit_table@@3U_onexit_table_t@@A 0000000180005220     MSVCRT:utility.obj
 0003:00000240       GS_ExceptionRecord         0000000180005240     MSVCRT:gs_report.obj
 0003:000002e0       GS_ContextRecord           00000001800052e0     MSVCRT:gs_report.obj
